:020000020000FC
:100000000C947125189518951895189518951895AC
:100010001895189518951895189518951895189578
:100020001895189518951895189518951895189568
:100030001895189518951895189518951895189558
:100040001895189518951895189518951895189548
:100050000C94E40718951895189518951895189507
:100060001895189518951895189518951895189528
:100070001895189518951895189518951895189518
:100080001895189518951895189518951895189508
:1000900018951895189518951895189518951895F8
:1000A00018951895189518951895189518951895E8
:1000B00018951895189518951895189518951895D8
:1000C00018951895189518951895189518951895C8
:1000D00018951895189518951895189518951895B8
:1000E00018951895189518951895189518951895A8
:1000F0001895189518951895189518951895189598
:100100001895189518951895189518951895189587
:100110001895189518951895189518950C94C90761
:100120001895189518951895189518951895189567
:10013000189518950C9449071895189518951895C1
:100140001895189518951895189518951895189547
:100150001895189518951895189518951895189537
:100160001895189518951895189518951895189527
:10017000189518951895189590F90F3F90F90FBF9D
:10018000D300053FD30005BF0000803FFE98FFBDB0
:100190000000803F561A20BD67A029BD9C5775BD41
:1001A0006FD1A5BD4AC9D4BDF8C102BEE1D3533F4A
:1001B000F8C102BE4AC9D4BD6FD1A5BD9C5775BD5B
:1001C00067A029BD1F1F1F00000000001C1E1F1F6D
:1001D0001F1F1F1F1F1F1F1F1F1F1E1C00000000AF
:1001E000001F1F1F1F1F1F1F1F1F0F07070F1F1F8E
:1001F0001F1F1F1F00000000001F1F1F1F1F1F00C9
:10020000001F1F1F0500010403022020052020FFFE
:100210000007010403060007010603020506FF208C
:1002200020FF050700060302050700040302000083
:10023000012020FF05070104030205070103030253
:100240000507070420200507070403030507010429
:1002500020200000691D0E009418501A701A9B1A75
:10026000F41A3F1B731BAC1BE91B501C821CB41CF3
:10027000EE1C2D1D0000F7220E0026215F217421A7
:100280008921B2211B2246226D227E228F22A022AA
:10029000BF22D922EA220000DF240E000D234B23C7
:1002A000602375239E2303242C2451246224732469
:1002B0008424A724C124D2240001382B352B4528BF
:1002C0002B02282B11922A0B572A01B02A01282B26
:1002D00001282B01282B02B02A05442A01852A0176
:1002E000922A03602A02922A038E2AFB03E333D068
:1002F00000EE1EE22BD100EE1EE228D100EE1EE23F
:1003000025D103E328D000EE1EE220D103E323D061
:1003100000EB14E01BD102E01ED000EB14E016D17C
:1003200008E019D000EB14E011D101E014D000EE88
:100330001EE20CD100EE1EE209D100EE1EE206D153
:1003400006E009D000EB14E001D10CE004D000EB92
:1003500014E0FCD008958A93802FE4E4F6E0008155
:100360000F7B00830CE310E0F1D000916406007F66
:1003700000936406082F02950F7010916406102BED
:1003800010936406E4E4F6E00081006800830CE367
:1003900010E0DCD0E4E4F6E000810F7700830CE2AB
:1003A00011E0D4D000916406007F009364068F7042
:1003B00000916406082B00936406E4E4F6E00081F3
:1003C000006800830CE310E0C1D0E4E4F6E00081B3
:1003D0000F7700830CE211E0B9D0899108958A93D8
:1003E000802FE4E4F6E00081006400830CE310E079
:1003F000ADD000916406007F00936406082F02953B
:100400000F7010916406102B10936406E4E4F6E07C
:100410000081006800830CE310E098D0E4E4F6E08B
:1004200000810F7700830CE211E090D00091640608
:10043000007F009364068F7000916406082B009380
:100440006406E4E4F6E00081006800830CE310E059
:100450007DD0E4E4F6E000810F7700830CE211E048
:1004600075D0899108950E94F028C801A0E007C0C6
:10047000B0E0FC01EA0FFB1F0081B1DFA395B0E003
:10048000FC01EA0FFB1F0081002311F0A13180F372
:10049000E4E00C9401295FDF07EC14E2E4DF089547
:1004A0000BEC0093520008E000935000E1E5F0E00F
:1004B000008103FFFBCF03EC00935500E0E5F0E083
:1004C000008100610083E1E5F0E0008104FFFBCFE3
:1004D00008ED04BF04E000934000E0E5F0E0008197
:1004E0000E7F0083089500E00093010202E2009372
:1004F000020203E00093040201E00093200200E204
:1005000000932102E0E0F2E00081016000830895A1
:1005100001E00093280200E300932902089501E01E
:100520000093300208E30093310208950DE0009338
:10053000200300E40093210300E00093220300E580
:100540000093240300E7009328030895015010400E
:1005500098018901232BD1F708958A93802F03C036
:1005600008EE1DEF07D08A95082F802F0023C1F7D2
:10057000899108950150104098018901232BD1F7EA
:1005800008950E94EC28942F81E035C0482F50E058
:10059000440F551F440F551FFA01E552FB4D0080D3
:1005A000118022803380482F50E0440F551F440FA4
:1005B000551FFA01E152FB4D0082118222823382E3
:1005C000482F50E0440F551F440F551FFA01ED52BC
:1005D000FB4D0080118022803380482F50E0440F73
:1005E000551F440F551FFA01E952FB4D008211823D
:1005F000228233828A95813048F6EFEDF4E200835F
:10060000118322833383492F50E008E010E00E94D9
:10061000BF25F801E059FE4F4591559165917491C0
:10062000EFEDF4E200811181228133810E94742771
:10063000E7EDF4E2008311832283338381E061C01C
:10064000E0E7F1E0082F10E0000F111F000F111F6D
:10065000E00FF11F492F50E008E010E00E94BF2595
:10066000E00FF11F4591559165917491082F10E0AD
:10067000000F111F000F111FF801E152FB4D008107
:100680001181228133810E94742728013901E0E819
:10069000F1E0082F10E0000F111F000F111FE00FF5
:1006A000F11F492F50E008E010E00E94BF25E00F45
:1006B000F11F4591559165917491082F10E0000F3D
:1006C000111F000F111FF801E952FB4D008111812C
:1006D000228133810E947427A801B901820193010C
:1006E0000E945727E7EDF4E24081518162817381D6
:1006F0000E941327E7EDF4E2008311832283338302
:100700008395823008F49CCFE7EDF4E200811181FB
:1007100022813381E8E00C94FD280E94EC28942F7C
:1007200081E035C0482F50E0440F551F440F551F3E
:10073000FA01E551FB4D0080118022803380482F63
:1007400050E0440F551F440F551FFA01E151FB4D76
:100750000082118222823382482F50E0440F551FBD
:10076000440F551FFA01ED51FB4D0080118022808E
:100770003380482F50E0440F551F440F551FFA0196
:10078000E951FB4D00821182228233828A958130A9
:1007900048F6EFEEF4E20083118322833383492F7E
:1007A00050E008E010E00E94BF25F801E059FE4F3C
:1007B0004591559165917491EFEEF4E200811181BC
:1007C000228133810E947427E7EEF4E200831183D3
:1007D0002283338381E061C0E0E7F1E0082F10E07D
:1007E000000F111F000F111FE00FF11F492F50E0E4
:1007F00008E010E00E94BF25E00FF11F45915591E0
:1008000065917491082F10E0000F111F000F111F48
:10081000F801E151FB4D00811181228133810E9459
:10082000742728013901E0E8F1E0082F10E0000FFB
:10083000111F000F111FE00FF11F492F50E008E0BA
:1008400010E00E94BF25E00FF11F45915591659181
:100850007491082F10E0000F111F000F111FF801F5
:10086000E951FB4D00811181228133810E9474275F
:10087000A801B901820193010E945727E7EEF4E233
:1008800040815181628173810E941327E7EEF4E277
:1008900000831183228333838395823008F49CCFB5
:1008A000E7EEF4E20081118122813381E8E00C94CB
:1008B000FD280E94EC28942F81E035C0482F50E09D
:1008C000440F551F440F551FFA01E550FB4D0080A2
:1008D000118022803380482F50E0440F551F440F71
:1008E000551FFA01E150FB4D0082118222823382B2
:1008F000482F50E0440F551F440F551FFA01ED508B
:10090000FB4D0080118022803380482F50E0440F3F
:10091000551F440F551FFA01E950FB4D008211820B
:10092000228233828A95813048F6EFEFF4E2008329
:10093000118322833383492F50E008E010E00E94A6
:10094000BF25F801E059FE4F45915591659174918D
:10095000EFEFF4E200811181228133810E9474273C
:10096000E7EFF4E2008311832283338381E061C0E7
:10097000E0E7F1E0082F10E0000F111F000F111F3A
:10098000E00FF11F492F50E008E010E00E94BF2562
:10099000E00FF11F4591559165917491082F10E07A
:1009A000000F111F000F111FF801E150FB4D0081D6
:1009B0001181228133810E94742728013901E0E8E6
:1009C000F1E0082F10E0000F111F000F111FE00FC2
:1009D000F11F492F50E008E010E00E94BF25E00F12
:1009E000F11F4591559165917491082F10E0000F0A
:1009F000111F000F111FF801E950FB4D00811181FB
:100A0000228133810E947427A801B90182019301D8
:100A10000E945727E7EFF4E24081518162817381A0
:100A20000E941327E7EFF4E20083118322833383CC
:100A30008395823008F49CCFE7EFF4E200811181C6
:100A400022813381E8E00C94FD280E94EE28542E88
:100A500080E090E0A0E0B0E04AE0442E1BC0442DCE
:100A600050E0440F551F440F551FFA01ED5FFA4D3A
:100A70000080118022803380442D50E0440F551FA8
:100A8000440F551FFA01E95FFA4D0082118222825C
:100A900033824A9441E0441610F7E7E0F5E2008320
:100AA00011832283338344242CC0ECE6F1E0042D2F
:100AB00010E0000F111F000F111FE00FF11F452D57
:100AC00050E00CE210E00E94BF25E00FF11F4591BD
:100AD000559165917491042D10E0000F111F000FC6
:100AE000111FF801E95FFA4D0081118122813381E4
:100AF0000E947427AC01BD010E941327C801D901CF
:100B000043940BE0401688F28C019D01E6E00C94C2
:100B1000FF280E94EE28542E80E090E0A0E0B0E094
:100B20004AE0442E1BC0442D50E0440F551F440F93
:100B3000551FFA01E15DFA4D00801180228033805B
:100B4000442D50E0440F551F440F551FFA01ED5C32
:100B5000FA4D00821182228233824A9441E0441687
:100B600010F7E3E3F5E20083118322833383442407
:100B70002CC0ECE6F1E0042D10E0000F111F000F77
:100B8000111FE00FF11F452D50E00CE210E00E9414
:100B9000BF25E00FF11F4591559165917491042D8A
:100BA00010E0000F111F000F111FF801ED5CFA4D4E
:100BB00000811181228133810E947427AC01BD0123
:100BC0000E941327C801D90143940BE0401688F214
:100BD0008C019D01E6E00C94FF280E94EE28542E23
:100BE00080E090E0A0E0B0E04AE0442E1BC0442D3D
:100BF00050E0440F551F440F551FFA01E55AFA4DB6
:100C00000080118022803380442D50E0440F551F16
:100C1000440F551FFA01E15AFA4D008211822282D7
:100C200033824A9441E0441610F7EFE5F5E2008381
:100C300011832283338344242CC0ECE6F1E0042D9D
:100C400010E0000F111F000F111FE00FF11F452DC5
:100C500050E00CE210E00E94BF25E00FF11F45912B
:100C6000559165917491042D10E0000F111F000F34
:100C7000111FF801E15AFA4D00811181228133815F
:100C80000E947427AC01BD010E941327C801D9013D
:100C900043940BE0401688F28C019D01E6E00C9431
:100CA000FF280E94EC28842FA52F0E94B426482FED
:100CB00050E0440F551F440F551FFA01E557FA4DF8
:100CC00040815181628173810E9457272801390137
:100CD0000A2F10E020E030E00E94BF26A801B901F1
:100CE000820193010E94ED27482F50E0440F551FC9
:100CF000440F551FFA01E557FA4D40815181628139
:100D000073810E94132790E0880F991F880F991F05
:100D1000FC01E557FA4D0083118322833383E8E019
:100D20000C94FD281091480001E0009348002091A8
:100D3000A0003091A2000091A2000C7F04600093FB
:100D4000A2004FB77894E8E4F0E0008101600083EE
:100D50005091CD01EF93FF930F932F93EBECF1E0C4
:100D600008ED21E004BF20832F910F91FF91EF91B7
:100D700003E00093CD018895109348002093A000D4
:100D80003093A2005093CD014FBF0895EFECF1E0F6
:100D9000008107FDFBCF0895F9DFEFECF1E0008162
:100DA00001FF11C006E30093CA01EF93FF930F9375
:100DB0002F93EBECF1E008ED21E004BF20832F91AD
:100DC0000F91FF91EF9108959A938A93C801DEDF06
:100DD0008B3000E0900748F04091E52750E000E4B8
:100DE00010E00E94BF25800F911F082F0093C001C3
:100DF000892F8F718093C10100E00093C20106E04A
:100E00000093CA01EF93FF930F932F93EBECF1E064
:100E100008ED21E004BF20832F910F91FF91EF9106
:100E20000091C4018991999108950E94F128C80107
:100E3000A22F00E00093060900E0009346088B30E3
:100E400000E0900748F04091E52750E000E410E012
:100E50000E94BF25800F911F9FDF03E30093CA010B
:100E6000082F0093C001892F8F718093C10100E08A
:100E70000093C201A093C40105E30093CA0152DFAD
:100E800003E00093060901E000934608E3E00C94B8
:100E900002299A938A93FA93EA930A927A936A932D
:100EA0005A934A933A932A931A930A930FB6E0E01F
:100EB000F2E00081046000830091BE2703950F706B
:100EC0000093BE270091C127002399F100912B27A1
:100ED00010912C27212F220F220B322F4091BE2759
:100EE00050E0440F551F440F551FFA01E553F94DCB
:100EF0004081518162817381400F511F621F731FB6
:100F0000408351836283738380913B2790913C2778
:100F1000019680933B2790933C27803004E0900714
:100F200041F400E00093C12710E000933B271093A9
:100F30003C270091BE2710E0000F111FF801E55378
:100F4000FA4D008111810093380310933903E5E2D3
:100F5000F3E0008101FF0EC00091BE2710E0000FFA
:100F6000111FF801E551FA4D0081118100933A03F8
:100F700010933B030FBE0991199129913991499121
:100F80005991699179910990E991F9918991999192
:100F900018954A933A932A931A930A934FB700915C
:100FA0001002109111022091DF273091E027021BDF
:100FB000130B00932B2710932C274FBF09911991E6
:100FC00029913991499118957A926A925A924A9246
:100FD0009A938A93FA93EA933A922A921A920A92ED
:100FE0007A936A935A934A933A932A931A930A9359
:100FF0009FB70091C127002309F08CC30091D5272A
:10100000033041F000E01091C727112319F400606C
:10101000002321F006E00093D72703C004E00093EB
:10102000D72780E033C05091D727482F642F082F4F
:1010300010E0000F111F000F111FF801E553F94DCB
:10104000008111812281338142E00E942726462FB0
:1010500028DE0E94C126282F30E0220F331FF9011D
:10106000E55FF84D0083118300E010E020E030E000
:10107000482F50E0440F551F440F551FFA01E55308
:10108000F94D00831183228333838395803158F295
:101090000FEF0093C12700E010E020E030E0E5E42E
:1010A000F7E20083118322833383E1E4F7E20083D4
:1010B000118322833383EDE3F7E2008311832283DC
:1010C000338300E010E020E030E0E1EEF7E200835F
:1010D00011832283338380E0CFC0082F10E0000FFC
:1010E000111FF801E55FF84D00811181212F220FBA
:1010F000220B322F0E94B42628013901082F10E05C
:10110000000F111FF801E55FF84D00811181212FBB
:10111000220F220B322F0E94B426A201B3010E949B
:101120007427E1EEF7E240815181628173810E9470
:101130001327E1EEF7E20083118322833383EDE38B
:10114000F7E200811181228133810E94B4262801B7
:101150003901082F10E0000F111FF801E55FF84D6D
:1011600000811181212F220F220B322F0E94B426E1
:10117000482F50E0440F551F440F551FFA01E55FFB
:10118000F94D40815181628173810E947427A201CF
:10119000B3010E9413270E94C126EDE3F7E200830A
:1011A000118322833383E1E4F7E2008111812281FC
:1011B00033810E94B42628013901082F10E0000F66
:1011C000111FF801E55FF84D00811181212F220FD9
:1011D000220B322F0E94B426482F50E0440F551F97
:1011E000440F551FFA01E55BF94D40815181628141
:1011F00073810E947427A201B3010E9413270E94E9
:10120000C126E1E4F7E20083118322833383E5E41E
:10121000F7E200811181228133810E94B4262801E6
:101220003901082F10E0000F111FF801E55FF84D9C
:1012300000811181212F220F220B322F0E94B42610
:10124000482F50E0440F551F440F551FFA01E55732
:10125000F94D40815181628173810E947427A201FE
:10126000B3010E9413270E94C126E5E4F7E2008340
:101270001183228333838395803108F42ECF40E09D
:1012800050E060E871E4E1EEF7E200811181228133
:1012900033810E94ED270E94582DE1EEF7E2008392
:1012A000118322833383E1EEF7E2008111812281F1
:1012B00033810E94C12648E050E00E94EB25009354
:1012C000DD271093DE27EDE3F7E200811181228113
:1012D0003381E1E5F7E20083118322833383E1E484
:1012E000F7E20081118122813381E5E5F7E2008395
:1012F000118322833383E5E4F7E2008111812281A7
:101300003381EDE5F7E2008311832283338300917B
:10131000C027002339F100E00093C027E1E5F7E2A0
:101320000081118122813381E5E6F7E20083118398
:1013300022833383E5E5F7E2008111812281338145
:10134000E1E6F7E20083118322833383EDE5F7E2E0
:101350000081118122813381E9E6F7E20083118364
:1013600022833383E5E6F7E2008111812281338114
:10137000E1E5F7E24081518162817381401B510BAD
:10138000620B730B4083518362837383E1E6F7E260
:101390000081118122813381E5E5F7E240815181AD
:1013A00062817381401B510B620B730B408351832D
:1013B00062837383E9E6F7E2008111812281338140
:1013C000EDE5F7E24081518162817381401B510B51
:1013D000620B730B40835183628373830091C72731
:1013E000002309F077C00091D5270330B9F541E01B
:1013F000E1E5F7E200811181228133810E94B42668
:1014000024DB0E94C126E9E8F7E2008311832283EE
:10141000338341E0E5E5F7E20081118122813381E8
:101420000E94B42676DB0E94C126EDE8F7E2008335
:1014300011832283338341E0EDE5F7E200811181DE
:10144000228133810E94B426C8DB0E94C126E5E8D0
:10145000F7E2008311832283338360C04091D52754
:10146000E1E5F7E200811181228133810E94B426F7
:101470000E94C1020E94C126E9E8F7E200831183BD
:10148000228333834091D527E5E5F7E2008111817E
:10149000228133810E94B4260E948D030E94C126BE
:1014A000EDE8F7E200831183228333834091D5274F
:1014B000EDE5F7E200811181228133810E94B4269B
:1014C000F8D90E94C126E5E8F7E200831183228360
:1014D000338324C0E1E5F7E2008111812281338169
:1014E000E9E8F7E20083118322833383E5E5F7E23D
:1014F0000081118122813381EDE8F7E200831183BD
:1015000022833383EDE5F7E200811181228133816B
:10151000E5E8F7E200831183228333830091D0272B
:1015200000950093D0270091D027002309F0CDC06B
:10153000E9E8F7E20081118122813381E5E9F7E2F0
:101540004081518162817381040F151F261F371F4F
:10155000E1EAF7E20083118322833383EDE8F7E2C7
:101560000081118122813381E9E9F7E240815181D3
:1015700062817381040F151F261F371FE5EAF7E20A
:101580000083118322833383E5E8F7E20081118130
:1015900022813381E1E9F7E24081518162817381E7
:1015A000040F151F261F371FEDE9F7E20083118393
:1015B000228333830091D12700950093D127009196
:1015C000D127002309F05CC084E00091D827801B5C
:1015D000E1EAF7E20081118122813381E9EAF7E251
:1015E0004081518162817381040F151F261F371FAF
:1015F000482F50E060E070E00E945226E9E4F7E2F4
:101600000083118322833383E5EAF7E200811181AD
:1016100022813381EDEAF7E2408151816281738159
:10162000040F151F261F371F482F50E060E070E0A1
:101630000E945226EDE4F7E2008311832283338374
:10164000EDE9F7E20081118122813381E1EBF7E2DC
:101650004081518162817381040F151F261F371F3E
:10166000482F50E060E070E00E945226E9E5F7E282
:1016700000831183228333830FEF0093D22750C05E
:10168000E1EAF7E20081118122813381E9EAF7E2A0
:101690000083118322833383E5EAF7E2008111811D
:1016A00022813381EDEAF7E20083118322833383C1
:1016B000EDE9F7E20081118122813381E1EBF7E26C
:1016C00000831183228333832BC0E9E8F7E2008192
:1016D000118122813381E5E9F7E2008311832283BE
:1016E0003383EDE8F7E20081118122813381E9E95A
:1016F000F7E20083118322833383E5E8F7E2008178
:10170000118122813381E1E9F7E200831183228391
:10171000338306C008E210E0009366081093670860
:101720009FBF0991199129913991499159916991D5
:1017300079910990199029903990E991F9918991BD
:101740009991499059906990799018950E94F02844
:1017500000E40E94AB01AFEF80E002C0A695839544
:101760008830A8F4BA2F90E005C000E00E94EF0195
:10177000B6959395983090F7BB2311F001E001C026
:1017800000E0002391F70FE10E94EF01F1CFE4E0C8
:101790000C9401299A938A9300E40E94AB0180E0A3
:1017A00008C090E0FC01EC53FE4F04910E94EF0151
:1017B00083958034B0F38991999108950E94F0281F
:1017C000D80180E090E02FC006E110E0AC010E945B
:1017D000BF250A0F1B1F212F220F220B322F0E9421
:1017E000B42640E050E064EB73E40E948E2830F4AD
:1017F00040E050E064EB73EC0E94132745E35AEF9E
:101800006EE87CE30E9474270E946D25AC01440FB2
:10181000551F440F551FFA01E557F94D00831183F9
:10182000228333830196803100E090076CF2E4E07C
:101830000C9401290E94F028D80180E090E02FC08C
:1018400006E110E0AC010E94BF250A0F1B1F212FEB
:10185000220F220B322F0E94B42640E050E064EBAE
:1018600073E40E948E2830F440E050E064EB73ECA7
:101870000E94132745E35AEF6EE87CE30E94742729
:101880000E948A2CAC01440F551F440F551FFA01CA
:10189000E55FF94D00831183228333830196803104
:1018A00000E090076CF2E4E00C9401290E94F0281B
:1018B000D80180E090E02FC006E110E0AC010E946A
:1018C000BF250A0F1B1F212F220F220B322F0E9430
:1018D000B42640E050E064EB73E40E948E2830F4BC
:1018E00040E050E064EB73EC0E94132745E35AEFAD
:1018F0006EE87CE30E9474270E946D25AC01440FC2
:10190000551F440F551FFA01E55BF94D0083118304
:10191000228333830196803100E090076CF2E4E08B
:101920000C9401290E94EC28D80180E090E034C09A
:101930008D01212F220F220B322F0E94B426280165
:1019400039018C01212F220F220B322F0E94B42645
:1019500049E058E964EC7EE30E9474270E948A2CD7
:10196000A201B3010E947427280139018D01212FA2
:10197000220F220B322F0E94B426A201B3010E9433
:1019800013270E94C1269C01220F331FF901E55144
:10199000FA4D008311830196803100E0900744F2F4
:1019A000E8E00C94FD280E94EA284801D90180E073
:1019B00090E046C006E110E0AC010E94BF25A801FE
:1019C000480D591D483601E0500714F04856514063
:1019D0008D01212F220F220B322F0E94B4262801C5
:1019E00039018A01212F220F220B322F0E94B426A7
:1019F0000801190145E35AEF6EE87CE3800191018B
:101A00000E9474270E948A2CA201B3010E947427AD
:101A1000280139018D01212F220F220B322F0E9424
:101A2000B426A201B3010E9413270E94C1269C0183
:101A3000220F331FF901E553FA4D008311830196FC
:101A4000803100E090070CF4B5CFEAE00C94FB285D
:101A50000E94F0282091BC273091BD270091BA2721
:101A60001091BB27A0DF6AD106E00E94AD02E09191
:101A7000DD27F091DE27F3970CF4F1C080E09CE5C0
:101A8000A1ECB7E400E010E00093EA271093EB2705
:101A900008C0EAEEF7E200811181065F1F4F008364
:101AA00011830091EA271091EB27083621E01207F5
:101AB000BCF520916D2430916E240091EA2710919D
:101AC000EB2771DF04E00E94AD020091DD27109149
:101AD000DE27212F220F220B322F0E94B426AC01C9
:101AE000BD010E947628A8F60091DD271091DE271F
:101AF000212F220F220B322F0E94B426C801D901B8
:101B00000091EA271091EB270093E6271093E7272F
:101B1000E091DD27F091DE27B8970CF0BACF54C0E2
:101B200080E09CE5A1ECB7E40AE010E0ADD000E075
:101B300010E000936D2410936E2408C0EDE6F4E2EB
:101B400000811181025E1F4F0083118300916D247B
:101B500010916E24083E27E01207B4F520916D2401
:101B600030916E240091E6271091E7271CDF04E0F6
:101B70000E94AD020091DD271091DE27212F220F58
:101B8000220B322F0E94B426AC01BD010E947628A0
:101B9000A8F60091DD271091DE27212F220F220BBE
:101BA000322F0E94B426C801D90100916D241091F2
:101BB0006E240093E8271093E927E091DD27F09148
:101BC000DE2774970CF0BACFE091E627F091E72773
:101BD0003B9744F0E6EEF7E2008111810850104097
:101BE00000831183E091E827F091E927759744F08D
:101BF000E8EEF7E2008111810F501040008311835D
:101C00002091E8273091E9270091E6271091E727F6
:101C1000CADE0091E8271091E9270093BC271093B2
:101C2000BD270091E6271091E7270093BA2710936C
:101C3000BB273091BB27232F00E210E0F6D820917C
:101C4000BA2701E210E0F1D83091BD27232F02E23C
:101C500010E0EBD82091BC2703E210E0E6D80FEFAC
:101C60000093BF27E4E00C94012934E0309340094D
:101C70003091D327329F00926A0910926B0900932A
:101C8000660910936709089524E044E650E00E9435
:101C9000BF25EBDF48E750E000912F271091302758
:101CA0000E94EB250E94AD0200E0009340090895D8
:101CB0000E94F128C801A22F04E00093400943E0EC
:101CC0000091D3270E94A125E02FF0E031964A2F02
:101CD00050E08F010E94BF2500936A0910936B09A1
:101CE0008093660990936709E3E00C9402298A9334
:101CF000812F10E0C9DF00E513EC0E94BA02082F23
:101D000010E0C2DF899108950E94F028D80181E097
:101D100090E00DC044E050E08C010E94EB25202FA4
:101D20008D01A3DF00E41CE90E94BA020196843110
:101D300000E090077CF3E4E00C94012924E231E216
:101D400007EC14E20E943D2D00E80E944B0200E3E4
:101D500010E09ADF08950E94052540E050E064E617
:101D600072E40E9474270E94C12608950E94EC2804
:101D7000D80125E331E207EC14E20E943D2D00E892
:101D80000E944B02A13000E0B00714F180E0082F60
:101D900010E020E030E00E94BF26280139018D01CB
:101DA000212F220F220B322F0E94B4260E940A29D3
:101DB000A801B901820193010E94762878F5082FC5
:101DC00007570E94AB010EE30E94EF018395DFCF1E
:101DD00080E008C006E8081B0E94AB010CE30E94EB
:101DE000EF018395082F10E020E030E00E94BF262D
:101DF000280139010FEF1FEFAD010E94BF25212FF0
:101E0000220F220B322F0E94B4260E940A29A80119
:101E1000B901820193010E947628E0F200E315E700
:101E20000E94BA02E8E00C94FD289A938A9300E09D
:101E300010E080E090E019C0E0E0F2E0208128604E
:101E4000208320912B022223E1F321E020932B0217
:101E50002091120230911302020F131F0A5B1040EF
:101E6000112312F400E010E00196803A20E092077E
:101E70001CF34DE450E00E94EB258991999108955F
:101E8000E0E0F2E000810061008300913302002372
:101E9000E1F301E0009333024091CD2750E000913F
:101EA0001402109115020E94D32508950091B627BF
:101EB0001091B727BFDC0091B6271091B727F6DC49
:101EC0000091B6271091B7270093B8271093B92730
:101ED0000091B8271091B92771DC08950091B627B9
:101EE0001091B727A7DC0091B6271091B727DEDC49
:101EF0000091B8271091B92761DC4091D92750E0B3
:101F00000FEF10E00E94BF250DDD00912F271091EB
:101F10003027009326091093270908959A938A93EE
:101F200000E110E00E94E406902F80E001E110E063
:101F30000E94E40610E0802B912B80932F27909332
:101F4000302706E110E00E94E406902F80E007E1D0
:101F500010E00E94E40610E0802B912B8093B627BE
:101F60009093B72708E110E00E94E406902F80E0EC
:101F700009E110E00E94E40610E0802B912B809391
:101F8000B8279093B92700E210E00E94E406902F52
:101F900080E001E210E00E94E40610E0802B912B2B
:101FA0008093BA279093BB2702E210E00E94E406D8
:101FB000902F80E003E210E00E94E40610E0802B06
:101FC000912B8093BC279093BD2702E110E00E94E3
:101FD000E4060093CA2703E110E00E94E4060093A0
:101FE000CB2705E110E00E94E4060093CC2704E231
:101FF00010E00E94E4060093D6270EE110E00E9454
:10200000E4060093D9270FE110E00E94E406009354
:10201000D52709E010E00E94E4060093CE270AE0ED
:1020200010E00E94E4060093CD2705E210E00E9434
:10203000E4060093D32706E210E00E94E406009332
:10204000DA270BE010E00E94E4060093D42707E2B1
:1020500010E00E94E40603700093D8270CE110E022
:102060000E94E406802F90E00DE110E00E94E4065B
:10207000102F00E0802B912B8093DB279093DC279F
:10208000EBEDF7E20081118101601068008311839C
:102090008991999108950E94F028D8010091C7274D
:1020A000002311F088E40DC0BB2312F48CE309C0B7
:1020B0004AE050E08D010E94EB25102F06E0109FB2
:1020C000802D00E80E94AB0190E0FC01EC5FFD4F29
:1020D00004910E94EF0101E80E94AB0190E0FC0135
:1020E000EB5FFD4F04910E94EF0102E80E94AB01FB
:1020F00090E0FC01EA5FFD4F04910E94EF0100ECCB
:102100000E94AB0190E0FC01E95FFD4F04910E9449
:10211000EF0101EC0E94AB0190E0FC01E85FFD4F94
:1021200004910E94EF0102EC0E94AB0190E0FC01DF
:10213000E75FFD4F04910E94EF010091C727002344
:1021400011F088E40CC0BB2312F482E408C04AE01A
:1021500050E08D010E94EB2506E0409F802D04E8B1
:102160000E94AB0190E0FC01EC5FFD4F04910E94E6
:10217000EF0105E80E94AB0190E0FC01EB5FFD4F31
:1021800004910E94EF0106E80E94AB0190E0FC017F
:10219000EA5FFD4F04910E94EF0104EC0E94AB0145
:1021A00090E0FC01E95FFD4F04910E94EF0105EC16
:1021B0000E94AB0190E0FC01E85FFD4F04910E949A
:1021C000EF0106EC0E94AB0190E0FC01E75FFD4FE0
:1021D00004910E94EF0103E80E94AB0100E20E941B
:1021E000EF0103EC0E94AB0100E20E94EF01E4E08A
:1021F0000C9401290E94E4282597F8940E9450022B
:10220000E0E8F6E0008108600083009160060F605E
:102210000093600600914006006C00934006E0E6E3
:10222000F6E0008100620083E0E4F6E000810260F5
:10223000008300916006006C0093600608E1009343
:10224000110608E10093120608E10093130608E165
:10225000009330060E94760108E010E00E94E40638
:102260000F3F11F401E001C000E0E8E0F6E010816A
:1022700011FD09C0E8E0F6E0108112FD02C011E096
:1022800003C010E001C010E0012B002309F4A3C03B
:1022900000E00093E5270FC02AE20A2F10E0085D56
:1022A0001F4F0E941507A395AB30B0F30091E527AF
:1022B00003950093E5270091E527043008F086C0D8
:1022C00026E431E207EC14E20E943D2D00E80E9472
:1022D0004B0208E20E94AD0221E000E110E00E9402
:1022E000150726E701E110E00E94150720E006E14E
:1022F00010E00E94150728E207E110E00E94150790
:1023000020E008E110E00E94150728E209E110E052
:102310000E94150720E000E210E00E94150720E06F
:1023200001E210E00E94150720E002E210E00E94A6
:10233000150720E003E210E00E94150722E002E109
:1023400010E00E94150728E003E110E00E94150745
:1023500020E005E110E00E94150725E00EE110E005
:102360000E94150722E00FE110E00E94150721E00E
:1023700004E210E00E94150720E00CE110E00E944A
:10238000150720E00DE110E00E94150728EC09E098
:1023900010E00E94150725E30AE010E00E941507EF
:1023A00024E005E210E00E94150726E00BE010E0B3
:1023B0000E94150722E007E210E00E94150721E0C5
:1023C00006E210E00E941507A0E06ECF20E008E0D2
:1023D00010E00E94150708E010E00E94E406009358
:1023E000E5279CDD0091DA27023011F4D3D901C032
:1023F000ADD908E00093CB2704E00093CA2702E0A0
:102400000093D52703E20093010807E0009300083A
:1024100006E910E000932608109327088091D4273E
:1024200090E0019680932A0890932B0807E0009390
:10243000400804ED11E0009366081093670801E07E
:102440000093460801E00093000900912F271091A6
:102450003027009326091093270903E0009306090B
:102460000091A20007600093A2000E9496022091B2
:10247000BC273091BD270091BA271091BB2793DA72
:1024800004E414E000930C0210930D020E94730206
:1024900002E0009322020E948F020E9488021EDD49
:1024A00002E00E94AD0203E200934109009164063C
:1024B0000F730093640626E531E207EC14E20E94F4
:1024C0003D2D00EC0E944B0227E631E207EC14E2BE
:1024D0000E943D2D00E80E944B0200ED17E014DC45
:1024E00000EA1FE011DC00E41FE10EDC00ED17E064
:1024F0000BDC00E00093400900E00093400902E398
:102500000E94AD020091C8240B3469F60091C924E1
:10251000003549F60091CA240F3429F6009164066B
:10252000006C009364060091CE2710E0005A164F0D
:102530000093DF271093E0270091CC24023309F0A9
:10254000B2CF789428E731E207EC14E20E943D2DE7
:1025500000EC0E944B02A9E10A2FA02FAA950023AC
:1025600009F4C5C00091E52710E01A930A9329E801
:1025700031E207EC14E20E943D2D229600E80E9411
:102580004B0205E00E94AD02E8E0F6E0008102FDAA
:1025900017C00091E52703950093E527043018F054
:1025A00003E00093E5272091E52708E010E00E9472
:1025B000150702E310E068DBB1DC90DCAAE01BC089
:1025C000E8E0F6E0008101FD16C00091E5270A95DC
:1025D0000093E5270F3F19F400E00093E5272091D1
:1025E000E52708E010E00E94150702E310E04CDB4D
:1025F00095DC74DCAAE002EC0E94AB01EE2409C079
:102600000E2D10E0085D1F4F0E94E4060E94EF01AE
:10261000E3940BE0E016A0F3E8E0F6E0008103FDB0
:102620009BCF08E210E030DB0DE00E94AB01A0E49C
:1026300002E00093CF270EC00091CF2703950093AF
:10264000CF270D3018F00CE00093CF27A0E408E26C
:1026500010E01ADB0091CF2700540E94AB0105E087
:102660000E94AD02E8E0F6E0008102FFE5CFE8E07D
:10267000F6E0008101FD0FC00091CF270A9500937D
:10268000CF27023018F402E00093CF27A0E408E23D
:1026900010E0FADADFCFE8E2F6E0008100FD1AC0D0
:1026A000A3950A2FA02F0B3508F0A0E30A2F0E9454
:1026B000EF010091CF2700540E94AB0102E310E02C
:1026C000E3DA2A2F0091CF2710E00A5D1F4F0E9406
:1026D0001507C0CFE8E0F6E0008103FDBBCF009115
:1026E000CF27033008F4B6CF08E210E0CDDA0CE0D3
:1026F0000E94AB0100E310E0C7DAA9E198C000E056
:1027000010E010D928E735E00091BA271091BB27D7
:102710004AD902E00E94AD024AE050E00091DD2774
:102720001091DE270E94EB25C801823400E090075B
:102730003CF0FC01E154F040EE0FFF1F8E0F9F1F95
:102740009A938A932AE931E207EC14E20E943D2D24
:10275000229600E80E944B022BEA31E207EC14E2D9
:102760000E943D2D00EC0E944B02E8E2F6E0008161
:1027700000FFC5CF05E00E94AD022091BC2730913B
:10278000BD270091BA271091BB270DD94091D927B9
:1027900050E00FEF10E00E94BF25C4D805E00E9472
:1027A000AD0243DB280140912F27509130274F5F26
:1027B0005F4F652F660F660B762F00E01CE62CED51
:1027C00032E00E94522644E00E942726C8015A9215
:1027D0004A929A938A932CEB31E207EC14E20E941E
:1027E0003D2D249600E80E944B020091DD271091B8
:1027F000DE271A930A932CEC31E207EC14E20E94D4
:102800003D2D229600EC0E944B020091D82710E04B
:102810001A930A9328ED31E207EC14E20E943D2D51
:1028200022960AEC0E944B0202E00E94AD020A2F9F
:10283000A02FAA95002309F098CF0AE0401600E0E7
:102840005006ACF421EE31E207EC14E20E943D2D7B
:1028500000E80E944B0200ED10E016DA00EB10E0F9
:1028600013DA00ED10E010DA01E00E94AD020091F1
:10287000DD271091DE27093E23E01207ACF022EF9E
:1028800031E207EC14E20E943D2D00EC0E944B0265
:1028900000ED10E0F9D900EB10E0F6D900ED10E002
:1028A000F3D902E00E94AD0205E00E94AD0201E012
:1028B0000093C02700E00093CF270EEF0A8300E0CB
:1028C000098306E00093C82700E010E00093352755
:1028D000109336270093332710933427212F220F8C
:1028E000220B322FE9E5F7E2008311832283338341
:1028F000DD24CC24C39404E10E94AD0200E310E087
:10290000C3D903E00E94AD0200E310E0BDD900E0AE
:1029100008830E94760111C000916406006C009348
:10292000640600E20093B527E3940E2DE02E0536F1
:1029300020F0EE2400E0009340090091C527002319
:1029400041F000E01881112321F40060002309F414
:10295000CAC30091C727002309F0F3C1E9E4F7E2F5
:102960000081118122813381EDE6F7E2008311833A
:1029700022833383EDE4F7E20081118122813381E8
:10298000E9E7F7E20083118322833383E9E5F7E285
:102990000081118100932D2710932E270091CA27C3
:1029A00010E020912D2730912E27021713070CF0ED
:1029B00094C10091C427002309F08FC1EE2400E0E8
:1029C0000093C8270091C92703950093C927E1E721
:1029D000F7E20081118122813381EDE6F7E2408147
:1029E000518162817381401B510B620B730B4083D9
:1029F000518362837383EDE7F7E2008111812281C5
:102A00003381E9E7F7E24081518162817381401BA4
:102A1000510B620B730B4083518362837383EDE62A
:102A2000F7E20081118122813381EDE6F7E24081F6
:102A30005181628173810E94FF25C801D901E9E7B4
:102A4000F7E20081118122813381E9E7F7E24081D9
:102A50005181628173810E94FF25A801B9018C0117
:102A60009D01040F151F261F371F0E94B4260E94C8
:102A7000582D0E94C12643E00E94CD2538017720C1
:102A800042F422E104EF1EE7F0D800E21EE40E94C7
:102A9000BA02E9E7F7E200811181228133810E94C5
:102AA000B426A801B901CA01DB01EDE6F7E2008115
:102AB0001181228133810E94B426AC01BD014BD922
:102AC000009331271093322700912D2710912E2744
:102AD000212F220F220B322F0E94B4260E940A2996
:102AE0000E94C126802F889F800149E050E02091FC
:102AF000D32730E0421B530B0E94EB25802F8E5FC3
:102B00000B811C8120912D2730912E27021713074E
:102B10007CF40091312710913227009337271093CE
:102B20003827630100912D2710912E270B831C83DA
:102B3000E0913727F09138273197E63500E0F0072C
:102B400008F065C04AE050E000913127109132272B
:102B50000E94EB25402F4A5F0091DB271091DC2774
:102B60000E94CD250170002309F051C00091372744
:102B7000109138270093352710933627009331277B
:102B8000109332270091D627013031F4282F00E42A
:102B90001FE10E94350EA7C20091D627023001F531
:102BA000E0913127F0913227759734F4282F00EB0C
:102BB00016E30E94350E97C20091312710913227FB
:102BC000063420E0120734F0282F00E717E10E94B6
:102BD000350E89C2282F00E41FE10E94350E83C202
:102BE000282F822FAAE0B0E04AE050E00091312780
:102BF000109132270E94EB25AD01401B510B00EDD7
:102C000017E00E94BF25282F0E94350E6CC200914C
:102C1000CB27002309F467C21091322711230AF051
:102C200062C20091CB2710E020912D2730912E27F2
:102C3000021713070CF057C294E04CEE5FEF0091BF
:102C40003127109132270E94EB25901B492F0091CC
:102C5000DB271091DC270E94CD250170002309F0AD
:102C600042C20091312710913227009335271093EB
:102C7000362742E0082F0E94A125802F009131279E
:102C800010913227073E2FEF120734F0282F00EB68
:102C900016E30E94350E27C20091D6270430B9F4FE
:102CA000282F822FA6E1B0E04AE050E000913127C2
:102CB000109132270E94EB25AD01401B510B08EE0D
:102CC00013E00E94BF25282F0E94350E0CC2282F2A
:102CD00000E915E60E94350E06C200E010E0009300
:102CE0006A0910936B0900E010E0009366091093E5
:102CF000670900E000934009EDE6F7E200811181E9
:102D000022813381E1E7F7E2008311832283338359
:102D1000E9E7F7E20081118122813381EDE7F7E2F3
:102D2000008311832283338300E010E00B831C8334
:102D30000091C82703950093C82700E00093C92796
:102D4000D2C10091D527033041F000E01881112352
:102D500021F40060002309F4E0C042E050E060E0AC
:102D600070E0E9E4F7E200811181228133810E9461
:102D70005226EDE6F7E2008311832283338342E09B
:102D800050E060E070E0EDE4F7E200811181228123
:102D900033810E945226E9E7F7E200831183228300
:102DA000338342E050E060E070E0E9E5F7E2008163
:102DB0001181228133810E94522600932D27109386
:102DC0002E27EDE6F7E20081118122813381EDE6C5
:102DD000F7E240815181628173810E94FF25C80121
:102DE000D901E9E7F7E20081118122813381E9E726
:102DF000F7E240815181628173810E94FF25A80121
:102E0000B9018C019D01040F151F261F371F0E9459
:102E1000B4260E94582D0E94C12644E00E94CD2570
:102E2000380177204AF422E100E01DE70E94350EC8
:102E300000E513EC0E94BA02F3940F2DF02E01313D
:102E400020F001E00093C027FF240091C427002355
:102E500049F010E00091C427063021F010601123E2
:102E600009F441C100912D2710912E27212F220F07
:102E7000220B322F0E94B4260E940A290E94C126EA
:102E8000802F889F802DE9E7F7E200811181228160
:102E900033810E94B426A801B9014A015B01EDE625
:102EA000F7E200811181228133810E94B426A401BE
:102EB000B5010E94AB0E0093352710933627009181
:102EC000D6270130A1F40091352710913627073E0F
:102ED0002FEF120734F0282F08E51BE10E94580E4F
:102EE0001AC0282F00EF15E50E94580E14C0282F95
:102EF000222E20EE3EE2EDE6F7E2408151818A018A
:102F00004091D62750E00E94BF25201B310B89013C
:102F1000222D0E94580E6301E6C042E050E060E0BE
:102F200070E0E9E4F7E200811181228133810E949F
:102F30005226EDE6F7E2008311832283338342E0D9
:102F400050E060E070E0EDE4F7E200811181228161
:102F500033810E945226E9E7F7E20083118322833E
:102F6000338343E050E060E070E0E9E5F7E20081A0
:102F70001181228133810E9452260150104000931A
:102F80002D2710932E27EDE6F7E200811181228193
:102F90003381EDE6F7E240815181628173810E94C5
:102FA000FF25C801D901E9E7F7E2008111812281FB
:102FB0003381E9E7F7E240815181628173810E94A8
:102FC000FF25A801B9018C019D01040F151F261FC3
:102FD000371F0E94B4260E94582D0E94C12645E04A
:102FE0000E94CD2538010091CA2710E020912D279D
:102FF00030912E27021713070CF06AC00091C427E6
:10300000002309F065C00091C92703950093C927E3
:103010000E3631F401E00093C02700E00093C92789
:10302000EE2400E00093C82777204AF422E100E074
:103030001DE70E94350E00E513EC0E94BA020091D4
:103040002D2710912E27212F220F220B322F0E9485
:10305000B4260E940A290E94C126802F889F8001E1
:1030600049E050E02091D32730E0421B530B0E94EF
:10307000EB25802F8E5F0091C927043058F0282F50
:1030800000EE1EE240912D2750912E27041B150BB8
:103090000E94350E6301E9E7F7E200811181228188
:1030A00033810E94B426A801B901CA01DB01EDE613
:1030B000F7E200811181228133810E94B426AC01A4
:1030C000BD010E94AB0E00933527109336270BC02D
:1030D00000E00093400900E00093C9270091C82751
:1030E00003950093C8270091C8270C3D41F010E0DC
:1030F0000091C9270C3D19F01060112379F000E010
:1031000010E0009335271093362700933327109350
:103110003427CC24DD2401E00093C0270091C4278C
:10312000E2E5F2E00C949F288091352790913627B4
:1031300001E0C01600E0D0062CF080933327909376
:10314000342704C080913327909134270091DA27E7
:10315000023009F073C08C010E944B1008EE13E09E
:103160000E94BA028601212F220F220B322F0E94C9
:10317000B4260E940A290E94C126C8010091C827CE
:10318000053048F023E032E207EC14E20E943D2DC6
:1031900007EC0E944B020091C727002321F00EE3A9
:1031A000402E552403C006E0402E5524A0E008C060
:1031B0000A2F08530E94AB01042D0E94EF01A39532
:1031C000B0E0A817B907A4F30091B52710E01A934F
:1031D0000A930091D52710E01A930A930091CA2709
:1031E00010E01A930A930091CB2710E01A930A93E8
:1031F0002DE032E207EC14E20E943D2D289607E80C
:103200000E944B020E94400F28014AE050E08201D8
:103210000E94EB255A934A934AE050E082010E94B3
:10322000EB251A930A9328E132E207EC14E20E949C
:103230003D2D24960DE80E944B024BC4992352F079
:103240009A938A932FE132E207EC14E20E943D2D1B
:10325000229609C09A938A9326E232E207EC14E29E
:103260000E943D2D229600E80E944B020A81102FF9
:1032700013951A83002371F409810095098309814C
:10328000002329F44090DD275090DE2703C00E94E0
:10329000400F28018601212F220F220B322F0E947E
:1032A000B4260E940A290E94C126C801883000E085
:1032B000900711F48FEF90E004E80E94AB01082F13
:1032C0000E94EF01992352F42CE232E207EC14E25F
:1032D0000E943D2D04E80E944B021EC00091B527BC
:1032E00010E01A930A930091D52710E01A930A93DD
:1032F0000091CA2710E01A930A930091CB2710E09F
:103300001A930A932EE232E207EC14E20E943D2D5A
:10331000289605E80E944B0209810023B1F04AE09B
:1033200050E082010E94EB255A934A934AE050E014
:1033300082010E94EB251A930A932AE332E207ECFA
:1033400014E20E943D2D249609C05A924A9222E42A
:1033500032E207EC14E20E943D2D22960CE80E9416
:103360004B020091C727002309F052C00091C827E3
:10337000053048F028E731E207EC14E20E943D2DC9
:1033800000EC0E944B02A82FE0913127F0913227E8
:1033900031977CF00091312710913227045C1F4F48
:1033A0004AE050E00E94EB250093392710933A271A
:1033B00012C042E050E000913127109132270E9464
:1033C000EB250E5C1F4F4AE050E00E94EB25009376
:1033D000392710933A270091392700540E94AB01F6
:1033E000A13058F00091C827013020F007E00E947A
:1033F000EF0103C004E00E94EF0105EC0E94AB0165
:103400000FE20E94EF0100ED17E00E94BA0261C3D3
:1034100043E083010E94CD25C801833C01E0900771
:1034200034F400E099231AF00060002311F082ECDC
:1034300091E025E331E207EC14E20E943D2D00EC1F
:103440000E944B02A0E00FC00A2F07530E94AB015D
:103450000EE30E94EF0106EC0A1B0E94AB010CE395
:103460000E94EF01A3950A2F10E020E030E00E94B7
:10347000BF26480159018C01212F220F220B322F28
:103480000E94B4260E940A29A801B901840195016D
:103490000E947628C8F200EA1FE00E94BA0219C30F
:1034A0000091DD271091DE271A930A9328E432E277
:1034B00007EC14E20E943D2D229600E80E944B0288
:1034C0000091CE2710E01A930A932AE532E207EC26
:1034D00014E20E943D2D229600EC0E944B02F9C29C
:1034E0000E94400FC8014AE050E08C010E94EB2589
:1034F0005A934A934AE050E08C010E94EB251A93BC
:103500000A932CE632E207EC14E20E943D2D249649
:1035100000E80E944B020091CD2710E01A930A9315
:1035200020E832E207EC14E20E943D2D229600ECE6
:103530000E944B02CEC20E94150FC8019A938A9333
:1035400021E932E207EC14E20E943D2D229600E8C8
:103550000E944B0245E0E5E5F7E2008111812281FE
:1035600033810E9427263A932A931A930A9345E0BF
:10357000E1E5F7E200811181228133810E94272653
:103580003A932A931A930A9324EA32E207EC14E25C
:103590000E943D2D289606E80E944B0240912F275D
:1035A000509130274F5F5F4F652F660F660B762F68
:1035B00000E01CE62CED32E00E94522644E00E941E
:1035C00027263A932A931A930A9322EB32E207ECC6
:1035D00014E20E943D2D249600EC0E944B0200E66E
:1035E0001AEE0E94BA0275C20091DD271091DE2703
:1035F0001A930A9322EC32E207EC14E20E943D2D6A
:10360000229600E80E944B020091BC271091BD2732
:103610001A930A932DEC32E207EC14E20E943D2D3E
:10362000229609E80E944B020FED10E01A930A93CC
:103630000091BA271091BB271A930A930AEA10E067
:103640001A930A9326ED32E207EC14E20E943D2D14
:10365000269600EC0E944B020091BF27002321F424
:1036600009E80E94AB0103C009EC0E94AB010EE324
:103670000E94EF0100E315E70E94BA022AC240E26D
:1036800050E060E070E0EDE4F7E20081118122811A
:1036900033810E9452260E94B60E2AEE32E207ECD7
:1036A00014E20E943D2D00EC0E944B020FED10E051
:1036B0001A930A930091B6271091B7271A930A9389
:1036C0000AEA10E01A930A9325EF32E207EC14E2BB
:1036D0000E943D2D26960AEC0E944B0200E21EE459
:1036E0000E94BA02F6C101E008830FEF0093C727DA
:1036F00044E050E060E070E0E9E5F7E2008111812C
:10370000228133810E9452260E94B60E2FEF32E2B0
:1037100007EC14E20E943D2D00EC0E944B020FEDDD
:1037200010E01A930A930091B8271091B9271A93C1
:103730000A930AEA10E01A930A9325EF32E207ECA3
:1037400014E20E943D2D26960AEC0E944B0200EDE9
:1037500017E00E94BA02BDC100E008830091D327A0
:1037600010E01A930A932BE033E207EC14E20E9474
:103770003D2D229600E80E944B0223E133E207EC44
:1037800014E20E943D2D06E80E944B022EE133E236
:1037900007EC14E20E943D2D00EC0E944B02A0E0D9
:1037A00010C00A2F0A530E94AB010A2F0E94EF019A
:1037B000A83031F40EEC0E94AB010FEF0E94EF0134
:1037C000A3950091D3270A1760F703E00E94AD028A
:1037D00080C10091D627033019F48AE090E014C02C
:1037E0000091D627043059F48EE090E000912F2705
:1037F00010913027009326091093270905C0809166
:10380000D62790E0880F991F9A938A932FE233E28C
:1038100007EC14E20E943D2D229600E80E944B0224
:1038200023E133E207EC14E20E943D2D06E80E94FA
:103830004B0227E333E207EC14E20E943D2D00EC3B
:103840000E944B02A0E010C00A2F0A530E94AB0155
:103850000A2F0E94EF01A83031F40EEC0E94AB0158
:103860000FEF0E94EF01A3950091D6270A1760F78A
:1038700002E00E94AD020091D627053081F48EE56A
:1038800091E009C0809326099093270908EB1BE07B
:103890000E94BA020496883E03E090079CF319C187
:1038A0000091DA2710E01A930A9328E433E207EC38
:1038B00014E20E943D2D229600E80E944B022AE568
:1038C00033E207EC14E20E943D2D00EC0E944B0213
:1038D000A0E010C00A2F0A530E94AB010A2F0E94D9
:1038E000EF01A83031F40EEC0E94AB010FEF0E9403
:1038F000EF01A3950091DA270A1760F703E00E9411
:10390000AD02E7C00091D42710E01A930A932CE689
:1039100033E207EC14E20E943D2D229600E80E945B
:103920004B022EE733E207EC14E20E943D2D00EC3F
:103930000E944B02A0E010C00A2F0A530E94AB0164
:103940000A2F0E94EF01A83031F40EEC0E94AB0167
:103950000FEF0E94EF01A3950091D4270A1760F79B
:1039600003E00E94AD02B5C00E94150F1A930A939E
:1039700020E933E207EC14E20E943D2D229600E894
:103980000E944B0223E133E207EC14E20E943D2D3A
:1039900006E80E944B0226E933E207EC14E20E949B
:1039A0003D2D00EC0E944B02A0E010C00A2F0A53EC
:1039B0000E94AB010A2F0E94EF01A83031F40EECF7
:1039C0000E94AB010FEF0E94EF01A3950091D92750
:1039D0000A1760F703E00E94AD027BC00091DD276B
:1039E0001091DE271A930A9322E432E207EC14E2E4
:1039F0000E943D2D229600E80E944B0223E133E213
:103A000007EC14E20E943D2D06E80E944B0227EAD3
:103A100033E207EC14E20E943D2D00EC0E944B02C1
:103A2000A0E010C00A2F0A530E94AB010A2F0E9487
:103A3000EF01A83031F40EEC0E94AB010FEF0E94B1
:103A4000EF01A3950091D8270A1760F703E00E94C1
:103A5000AD0201E00093C2273CC00091C2270023C1
:103A6000C1F128EB33E207EC14E20E943D2D00E89F
:103A70000E944B02A0E004C000E20E94EF01A39567
:103A8000A03190F40A2F00540E94AB014A2F0091FC
:103A9000DB271091DC270E94CD250170002361F304
:103AA00003E20E94EF01EBCF05EC0E94AB010FE2B5
:103AB0000E94EF010091CF2700540E94AB010EE05D
:103AC0000E94AB0100E00093C22708EE1DEF0E94A8
:103AD000BA02B0E0E8E0F6E0008103FD85C000E056
:103AE0000093400901E00093C027E8E0F6E0008180
:103AF00003FD4BC008EE1DEF0E94BA02B3950B2FD9
:103B0000B02F003190F30091C52700950093C52791
:103B100001E00E94AB010091C5270023B1F400E051
:103B20000093C4274091D92750E00FEF10E00E9486
:103B3000BF250E94920C0091DA27023011F40E94F6
:103B4000CA0B03E00E94AD020CC007E00093C4273B
:103B500008E00E94AD0200E010E00E94920C0E947A
:103B6000A60B01E00093C22700E00093C62700E007
:103B70000093C7270AE510E00E94440E01E000937D
:103B8000C02703E00E94AD0258C10091C527002361
:103B900049F40091C72700950093C7270AEA0093CC
:103BA000C8271AC00CE00E94AB010091C4270395FE
:103BB0000093C4270E3018F001E00093C427009151
:103BC000C427083049F44091D92750E00FEF10E0A6
:103BD0000E94BF250E94920C08E210E00E94440E51
:103BE00005E00E94AD02F2C6E8E2F6E0008100FDC9
:103BF0001FC300E0009340090091C427005081F0EA
:103C00000A9509F424C1025009F460C10A9509F427
:103C1000A2C20A9509F4A2C1085009F4C2C200C3A5
:103C2000E8E2F6E0008100FDDCC008EE1DEF0E9436
:103C3000BA02B3950B2FB02F003190F300E310E0E0
:103C40000E94440EE5E5F7E2008111812281338173
:103C50000E94B426A801B901CA01DB01E1E5F7E23F
:103C600000811181228133810E94B426AC01BD0103
:103C70000E94AB0E0093312710933227E1E5F7E263
:103C80000081118122813381E5E7F7E2008311830E
:103C900022833383E5E5F7E20081118122813381BC
:103CA000E1E8F7E200831183228333838301212F2C
:103CB000220F220B322F0E94B4260E940A29409123
:103CC0003127509132275A934A9340E050E060E008
:103CD00070E40E9474270E94C1261A930A9329EC6B
:103CE00033E207EC14E20E943D2D249600E80E9486
:103CF0004B020091312710913227053C2FEF12071C
:103D000064F400E02091312730913227253A1FEFEB
:103D100031071CF00060002399F02EED33E207EC30
:103D200014E20E943D2D00EC0E944B0200EB10E0DB
:103D30000E94440EE8E2F6E0008100FFFBCF7DC068
:103D40002FEE33E207EC14E20E943D2D00EC0E94BE
:103D50004B0200E210E00E94440E8091B627909141
:103D6000B7270091312710913227801B910B8A557C
:103D7000904001968093B8279093B9271091B92766
:103D8000112342F4E8EBF7E20081118108591E4F3C
:103D9000008311830E946E0FE8E2F6E0008100FFCD
:103DA000FBCF01E00093C02728E731E207EC14E2E3
:103DB0000E943D2D00EC0E944B023091B927232F29
:103DC00008E110E00E9415072091B82709E110E0F2
:103DD0000E94150705E00E94AD0201E00093C02794
:103DE0002CC001E00093C0270091DD271091DE2751
:103DF0001A930A9320E034E207EC14E20E943D2D6E
:103E0000229600E80E944B0228E731E207EC14E218
:103E10000E943D2D00EC0E944B0200E310E00E9446
:103E2000440E0091C927002311F401E001C000E015
:103E30000093C8270CE00E94AD0221E134E207ECB8
:103E400014E20E943D2D00E80E944B02BFC50E9473
:103E50009E0E00E010E00E94920C08E8402E03E164
:103E6000502E80E090E01AC08C01005A164F00934B
:103E7000DF271093E02708EE1DEF0E94BA020091A1
:103E8000DD271091DE27041515053CF44090DD2751
:103E90005090DE27082F0093CE2703968B3F00E03B
:103EA000900714F32091CE2709E010E00E94150737
:103EB00010E600E40E94770E4091D92750E00FEF02
:103EC00010E00E94BF250E94920C80C5A0E0B0E0E7
:103ED0000E949E0E8EE591E012C080932609909379
:103EE000270905E00E94AD020E94150FA017B10737
:103EF0002CF4D80180932F27909330270496833F8A
:103F000001E0900754F300912F2710913027009380
:103F100026091093270910E400E50E94770E3091DE
:103F20003027232F00E110E00E94150720912F2752
:103F300001E110E00E94150749C529E334E207ECCE
:103F400014E20E943D2D00E80E944B0200E810E0C0
:103F50000E94440E00E810E00E94440EE8E2F6E001
:103F6000008100FDE2C000E61AEE0E94BA02B3959D
:103F70000B2FB02F053190F301E00093C32727E109
:103F800034E207EC14E20E943D2D00E80E944B024F
:103F900000E310E00E94440E01E00093C02708E215
:103FA0000E94AD0228E234E207EC14E20E943D2DAB
:103FB00000E80E944B0200E310E00E94440E0EE174
:103FC0000E94AD0280E090E0A0E01EC0E5E5F7E2CF
:103FD00000811181228133810E94B426A801B90198
:103FE0004A015B01E1E5F7E2008111812281338121
:103FF0000E94B426A401B5010E94AB0E800F911F50
:104000000BE00E94AD02A395AA3000F34AE050E015
:104010008C010E94EB25C801E091B627F091B727EB
:10402000EA55F040E81BF90BE093B627F093B72769
:104030000091B6271091B727093621E0120744F006
:10404000E6EBF7E2008111810856114000831183ED
:104050001091B727112342F4E6EBF7E200811181BA
:1040600008591E4F008311830E94560F0EE00E94D4
:10407000AD02E5E5F7E200811181228133810E94E2
:10408000B426A801B9014A015B01E1E5F7E200812C
:104090001181228133810E94B426A401B5010E94BE
:1040A000AB0E28010CEA40160FEF50060CF045CF7E
:1040B0002AE434E207EC14E20E943D2D00E80E945D
:1040C0004B0205E210E00E94440E05E00E94AD02A2
:1040D00005E210E00E94440E0091B6271091B72728
:1040E0000093B8271093B9270091B8271091B927EA
:1040F0000E94DE0B3091B727232F06E110E00E94CB
:1041000015072091B62707E110E00E9415073091AE
:10411000B927232F08E110E00E9415072091B82746
:1041200009E110E00E94150719CF0091C327002371
:1041300089F42BE534E207EC14E20E943D2D00E8FF
:104140000E944B0208EE1DEF0E94BA0200E510E04B
:104150000E94440E3BC4E8E2F6E0008100FD14C07A
:1041600008EE1DEF0E94BA02B3950B2FB02F053158
:1041700090F300E610E00E94440E0E94280D10E229
:1041800000E30E94770E59CE0091BF27009500935F
:10419000BF2702E310E00E94440E05E00E94AD023A
:1041A00015C481E090E04091CF278C010E94C72583
:1041B000C8014091CF270091DB271091DC270E9496
:1041C000CD250170002379F080959095EBEDF7E215
:1041D00000811181082319230083118310E500E475
:1041E0000E94770E0CC0EBEDF7E200811181082BE5
:1041F000192B0083118310E300E40E94770E01E085
:104200000093C2272091DB270CE110E00E941507E4
:104210003091DC27232F0DE110E00E941507D6C353
:1042200001E00093C02708E210E00E94440ECEC3D4
:10423000E8E0F6E0008102FDE2C100E00093400901
:104240000091C427E4E7F2E00C949F28E8E0F6E050
:10425000008102FD1FC000E61AEE0E94BA02B3956B
:104260000B2FB02F033190F30091CC2700950093D2
:10427000CC272091CC2705E110E00E94150701E032
:104280000093C32700E510E00E94440E01E00E9465
:10429000AD029FC30091C327002381F40091CA2778
:1042A00003950093CA270A3018F000E00093CA274C
:1042B0002091CA2702E110E00E94150798C10091E1
:1042C000CE2703950093CE270B3F18F000E0009314
:1042D000CE272091CE2709E010E00E94150700E4C8
:1042E0001CE90E94BA0283C10091CD270395009377
:1042F000CD270D3318F001E00093CD272091CD2775
:104300000AE010E00E94150700E41CE90E94BA02CE
:104310006EC180912F2790913027019780932F278E
:10432000909330278E3501E0900734F40EE511E0CC
:1043300000932F271093302700912F2710913027BB
:10434000009326091093270930913027232F00E18D
:1043500010E00E94150720912F2701E110E00E9434
:10436000150745C1E8E0F6E0008101FD11C000E05D
:1043700010E00093BC271093BD270093BA27109339
:10438000BB2704E610E00E94440E06E00E94AD0246
:104390000091BF27002309F58091BC279091BD278C
:1043A00001968093BC279093BD27813008E0900749
:1043B00034F000E018E00093BC271093BD27309143
:1043C000BD27232F02E210E00E9415072091BC2791
:1043D00003E210E00E94150720C08091BA27909157
:1043E000BB2701968093BA279093BB27893601E0BB
:1043F000900734F000E010E00093BA271093BB2739
:104400003091BB27232F00E210E00E941507209176
:10441000BA2701E210E00E9415072091BC273091D5
:10442000BD270091BA271091BB270E94D30C02E050
:104430000E94AD02DCC08091B6279091B72701960B
:104440008093B6279093B727883601E0900734F021
:1044500000E010E00093B6271093B7270E94560F94
:104460000091B6271091B7270093B8271093B9276A
:104470003091B727232F06E110E00E941507209105
:10448000B62707E110E00E941507B1C08091B82758
:104490009091B92701968093B8279093B9278836D1
:1044A00001E0900734F000E010E00093B82710938B
:1044B000B9270091B8271091B9270E94DE0B3091DF
:1044C000B927232F08E110E00E9415072091B82793
:1044D00009E110E00E9415078AC00091D3270395D7
:1044E0000093D327093018F008E00093D3272091D8
:1044F000D32705E210E00E94150779C00091D62766
:1045000003950093D627053018F004E00093D627D2
:104510002091D62704E210E00E94150768C00091A0
:10452000DA2703950093DA27033018F002E00093AE
:10453000DA272091DA2706E210E00E94150757C01B
:104540000091D42703950093D427093018F008E090
:104550000093D4270BE910E0009326081093270856
:104560002091D4270BE010E00E9415078091D427FA
:1045700090E0019680932A0890932B0838C0009110
:10458000D92703950093D927093018F008E0009344
:10459000D9274091D92750E00FEF10E00E94BF25A6
:1045A0000E94920C2091D9270EE110E00E9415077D
:1045B0001EC00091D82703950093D827043018F027
:1045C00003E00093D8272091D82707E210E00E944B
:1045D00015070DC00091CF2703950093CF27003119
:1045E00018F000E00093CF2701E00093C22708E213
:1045F00010E00E94440E01E00093C027E7C1E8E00C
:10460000F6E0008101FDE2C100E000934009009165
:10461000C427E6E9F2E00C949F28E8E0F6E0008188
:1046200001FD24C000E61AEE0E94BA02B3950B2FDA
:10463000B02F0E3090F30091D52703950093D52726
:10464000043018F001E00093D5272091D5270FE121
:1046500010E00E94150701E00093C32700E510E079
:104660000E94440E03E00E94AD02B3C10091C32733
:10467000002381F40091CB2703950093CB270A30C8
:1046800018F000E00093CB272091CB2703E110E046
:104690000E94150794C10091CE270A950093CE275A
:1046A0000E3F18F00AEF0093CE272091CE2709E0A5
:1046B00010E00E94150700E41CE90E94BA027FC1C5
:1046C0000091CD270A950093CD27002319F40CE320
:1046D0000093CD272091CD270AE010E00E94150716
:1046E00000E41CE90E94BA026AC180912F279091D0
:1046F0003027019680932F2790933027843F01E045
:10470000900734F003EF11E000932F271093302728
:1047100000912F2710913027009326091093270925
:1047200030913027232F00E110E00E9415072091DF
:104730002F2701E110E00E94150741C1E8E0F6E0F3
:10474000008102FD11C000E010E00093BC2710932F
:10475000BD270093BA271093BB2704E610E00E9400
:10476000440E06E00E94AD020091BF270023F9F439
:104770008091BC279091BD2701978093BC2790938F
:10478000BD27992332F400E010E00093BC2710937A
:10479000BD273091BD27232F02E210E00E941507AC
:1047A0002091BC2703E210E00E9415071EC08091F3
:1047B000BA279091BB2701978093BA279093BB2784
:1047C000992332F408E611E00093BA271093BB272F
:1047D0003091BB27232F00E210E00E9415072091A3
:1047E000BA2701E210E00E9415072091BC27309102
:1047F000BD270091BA271091BB270E94D30C02E07D
:104800000E94AD02DCC08091B6279091B727019736
:104810008093B6279093B727992332F408E611E0E6
:104820000093B6271093B7270E94560F0091B62722
:104830001091B7270093B8271093B9273091B72765
:10484000232F06E110E00E9415072091B62707E10B
:1048500010E00E941507B3C08091B8279091B92746
:1048600001978093B8279093B927992332F408E6EB
:1048700011E00093B8271093B9270091B827109141
:10488000B9270E94DE0B3091B927232F08E110E0F1
:104890000E9415072091B82709E110E00E94150732
:1048A0008EC00091D3270A950093D3270F3F19F4A8
:1048B00000E00093D3272091D32705E210E00E9467
:1048C00015077DC00091D6270A950093D6270130A1
:1048D00018F401E00093D6272091D62704E210E0D7
:1048E0000E9415076CC00091DA270A950093DA2719
:1048F000013018F401E00093DA272091DA2706E26C
:1049000010E00E9415075BC00091D4270A95009320
:10491000D4270F3F19F400E00093D4270091D42747
:10492000002331F400E010E00093260810932708DC
:104930002091D4270BE010E00E9415078091D42726
:1049400090E0019680932A0890932B0838C000913C
:10495000D9270A950093D9270F3F19F400E0009357
:10496000D9274091D92750E00FEF10E00E94BF25D2
:104970000E94920C2091D9270EE110E00E941507A9
:104980001EC00091D8270A950093D827013018F44B
:1049900001E00093D8272091D82707E210E00E9479
:1049A00015070DC00091CF270A950093CF270F3F21
:1049B00019F40FE00093CF2701E00093C22708E22B
:1049C00010E00E94440E01E00093C02700E0009335
:1049D000C3270091CE2710E0005A164F0093DF271F
:1049E0001093E0270091CC27002311F40C948C1431
:1049F000009164060F73009364060AE20093B527E2
:104A00000C94941400008895FECF0E94EC28C801F5
:104A1000D9012A013B015CD057D071F48201930186
:104A200053D051F401E2ECEEF7E2008341830FEF43
:104A30001FEF2FE73FE73DC044D0A201B3010E9422
:104A40001327AC01BD0140D061F442D03AD00E949E
:104A50008E280BED1FE029EC10F43FE32AC03FEB5A
:104A600028C0A201B3012DD00E94ED270801190131
:104A70002FD0820193010E94762823D0A0F41CD06D
:104A800050F424D0A801B9010BED1FE029E430E473
:104A90000E9457270EC01AD04BED5FE069E470EC1E
:104AA0000E94132706C008D010F410D002C00ED008
:104AB0003058E8E00C94FD280E948E288001910176
:104AC00008958C019D0108950C946C280C94EE2B94
:104AD00040E050E060E070E008953F7741E00C94E2
:104AE0008D2C03E20DBF01E20EBFC0E0D1E20E94B7
:104AF0008D29002311F00E94702C0E94FA100E9450
:104B000002250C9402250D01DA0140E050E060E03E
:104B100070E00E946C2839F400E010E04D934C9353
:104B200020E030E00CC0B901660F771F7E57572F89
:104B3000550F550B7D935C932F7730783F63D001F1
:104B400008950024E8E0EA9532F0001F001C0416E6
:104B5000D0F3041AF8CF001F402D00950895FF27C9
:104B6000442312F4F1604195002312F4F09501956D
:104B70000E94A125F0FD0195F1FD41950895149F36
:104B8000102D059F100D049F002D110D08954A95BD
:104B90001AF0000F111FFBCF08954A951AF01595D2
:104BA0000795FBCF089500241124EFE0001F111F8B
:104BB000001C111C0416150610F0041A150AEA95BB
:104BC000AAF7001F111FA001009510950895519597
:104BD000419550400895FF27552312F4F160F7DF07
:104BE000112312F4F09507D00E94D325F0FD03D0D5
:104BF000F1FDEDCF089511950195104008952224FF
:104C0000349F302D259F300D169F300D079F300D9E
:104C1000249F202D310D159F200D311D069F200D45
:104C2000311D149F102D210D321D059F100D211DCA
:104C3000321D049F002D110D221D321D08954A952D
:104C40002AF03695279517950795F9CF08954A9537
:104C50002AF03595279517950795F9CF08950024E3
:104C600011241001E0E2EA9592F0001F111F221FAB
:104C7000331F001C111C221C331C041615062606AB
:104C8000370688F3041A150A260A370AECCF001FE4
:104C9000111F221F331FA001B1010095109520950F
:104CA00030950895FF27772312F4F16015D0332350
:104CB00012F4F09509D00E942F26F69508F404D03E
:104CC000F69508F409C00895309520951095019542
:104CD0001F4F2F4F3F4F0895709560955095419508
:104CE0005F4F6F4F7F4F0895FF27112477FB660FAB
:104CF000771F089409F4771F679517F8EE270024AB
:104D000037FB220F331F089409F4331F279507F848
:104D1000089527FD0EC0EE0F001F111F221F3A95A8
:104D20003230B8F7332319F427FD31E002C027FFF2
:104D300030E0E03821F400FF08940EF488940F4F1F
:104D40001F4F2F4F3F4F323038F4332319F427FDD4
:104D500031E002C027FF30E03F3F29F0220F000C76
:104D6000379527950895ACC0032E002012F40E94B9
:104D70006426E02F012F122F232F3EE9D1CF0024EC
:104D8000F8CFBCDF432F4F5748F04F3148F007FCB6
:104D900091C03FE72FEF1FEF0FEF089533278CC02F
:104DA000322F212F102F0E2F4F5141950E941F2679
:104DB00007FE08950C946426F901EE0FFF1F37FBE0
:104DC000FF3F31F0EF2BE12BE02B8894B89408954E
:104DD000E02BE12B21F008949894B89408959894CE
:104DE000889438940895FB01EE0FFF1F77FBFF3F77
:104DF00031F0EF2BE52BE42B8894B8940895E42B45
:104E0000E52B69F3E8CFEFDF68F021F43723262F95
:104E10008A010895372FFBCFE6DF20F00BF00895CD
:104E20007327EAF751C0C8DFE8F3B3F361F3DBDFC0
:104E3000C8F383F3A1F358DF4017510762077307E4
:104E400031F4011411F10024E89488942BC078F017
:104E5000332E372F732D322E262F632D312E152F03
:104E6000532D302E042F432D302C012C132C3717AB
:104E700039F0669557954795F795E0407395F7CFCC
:104E8000E7FBEE0FE0E010246AF0EF0F041F151FA0
:104E9000261F60F4279517950795E79508F4689401
:104EA00033953ECFEF0B040B150B260B39CFE0E803
:104EB0007E27B9CF302D307822271127002708957B
:104EC0003FE7302920E8F9CF3FEF2FEFF6CF8BDF18
:104ED000D8F3D1F370783727089585DFA8F3A3F3CB
:104EE000F9CF3078372793CF67DF70F383F3A9F3D7
:104EF0007ADF50F3B3F3A9F3F7DE0124E8943F57C8
:104F0000E040370FEF1F12F0D9F603C03A3E90F29F
:104F10006894E0E00A92AA933A93AA2733242224C1
:104F20003327049FF001059FF00D712D731F149F0F
:104F3000F00D711D221C069F700D211C331C159F46
:104F4000700D211C331E249F700D211C331E169FD3
:104F5000200C311CAA1F259F200C311CA31F269F4B
:104F6000300CA11D39915EF43395A69537942794A2
:104F70007795F795E79533953130BCF316C0AA23A2
:104F800022F0332351F4339510C0339571F4A99175
:104F9000099096CFA7FD09C03A95EE0FFF1F771F26
:104FA000221C331CAA1F3230A8F7E894FE2B09F00C
:104FB00068942A2F8101E72FA9910990BACE13DFB7
:104FC00010F00BF087CF80CF0EDFE9F3E0F3032E74
:104FD000072670CF032E072673CFEEDEA0F37BF3F8
:104FE00099F301DF80F39BF3A9F37EDE012427FD13
:104FF00006C0000F111F221F3150E040F8CF67FD9F
:1050000006C0440F551F661F7150F040F8CFE8945A
:10501000371BEF0B3158EF4F2AF0EE23E9F63F3FF5
:10502000D9F203C03A3EA8F26894E0E0F0E011241F
:10503000139440175107620738F0315008F4689410
:10504000000F111F221FEE1F041B150B260BEF0B69
:10505000000F111F221FEE1F0A9279E17A95AAF024
:10506000041715072607EF0730F0041B150B260B56
:10507000EF0B089401C08894111C221C331C001CE7
:10508000000F111F221FEE1FE9CFF0F9E894E22B69
:10509000E12BE02B09F06894069437942794179439
:1050A000E79508F468947395B9F30990332311F0E8
:1050B000F0FF09C0369427941794E79508F4689494
:1050C00033953130BCF3012D122D232D32CE8BCEF2
:1050D00098940895189408956FDED0F3C1F383DE99
:1050E000B8F3041715072607370708957CDEA0F0EC
:1050F00063DE90F029F0E32FE7273AF47317089561
:1051000072DE51F04EF00894089504171507260733
:10511000370719F016F4B8F78894089564DEE0F3C1
:105120004BDED0F3E7DFC0F30894089575916591E5
:1051300055914591159011FA259035900895F9DF14
:10514000041B10E003C0F4DF041B150B20E030E06B
:1051500005C0ECDF041B150B260B370BB8F010FC59
:1051600017C045910590E00FF11F0417100540E0AE
:105170002407340758F436F404910024F101E01BAD
:10518000F0090994E00FF11F25903590F101099481
:1051900011F4D6F7F1CF31960EF0319650E060E081
:1051A00070E045914B3F48F089F34F3F29F04E3F67
:1051B00011F07591659155914591041B150B260BC6
:1051C000370B39F318F3E7CFFA92EA92DA92CA92E0
:1051D000BA92AA929A928A927A926A925A924A922F
:1051E000BA93AA939A938A930895FF84EE84DD84F8
:1051F000CC84BB84AA84998488847F806E805D80FF
:105200004C80BB81AA8199818881F0E0EC0FFD1F61
:10521000EF0108950E94E828229741E050E060E005
:1052200070E00E94762860F440E00E946C2821F42F
:1052300002E26BD03FEF5FC001E267D03FE75BC0A7
:10524000AE010E948325C801D90143EF54E065E314
:105250007FE30E94762868F437FBAA0FBB1FB39543
:10526000B695A795B7F908811981015010400883B8
:10527000198340E050E060E87FEB43D0280139011A
:1052800040E050E060E87FE33CD0A801B901820132
:1052900093010E94ED27C801D901A801B9012FD0BF
:1052A000280139010881102F110F110B212F312FE7
:1052B0000E94B42648E152E761E37FE320D0480131
:1052C000590142E252E964ED7EE38201930117D075
:1052D0004DED5BE96AE27FE316D0A201B3010FD086
:1052E00044E050E060E070E40ED0AC01BD0107D0B6
:1052F000A401B50108D02296ECE00C94F9280C9496
:1053000074278C019D010C941327ECEEF7E20083C7
:1053100051830FEF1FEF2FE7089501E008950E94DA
:10532000E428EF97EF976A972A873B874887598742
:1053300068017B0100E00B830C8302C011D21BD2F9
:105340000AD2053251F00023C9F70B811C81EF9678
:10535000EF966A96E0E10C94F5280081053221F47D
:1053600002D2FED105E2EBCF00E00F830E830A8369
:1053700009833E0102E1600E00E0701E0FE614E2B8
:10538000088B198B06C00981002311F40081098361
:10539000EAD1D9D10052B9F3035059F00850B1F312
:1053A000025019F0035049F00CC00A8103950A839A
:1053B000EFCF0E8103950E83EBCF0F8103950F8303
:1053C000E7CF00810A3279F4AAD1AD90BD9098D18F
:1053D000BB203AF4B194A19400E0B00A0A8103958D
:1053E0000A83C1D114C0AA24BB244AE050E00DC0F6
:1053F00021916F0185010E94BF25A22EBB24A00E22
:10540000B11E00EDA00E0FEFB01EA0D188F30A81EF
:10541000002311F000E00F8396D10E32F1F4A3D1F6
:1054200092D10A3231F47BD18D909D9069D19BD17C
:1054300017C0882499244AE050E088D188F421914B
:105440006F0184010E94BF25822E9924800E911E37
:1054500000ED800E0FEF901EF0CF88248A94982CD8
:1054600080E071D10C5421F00C5131F0045039F42A
:1054700081E0C80E7AD103C001E0C00ED81E6BD106
:10548000E8EBF2E00C949F2880FB5EF44B815C819A
:10549000652F660F660B47D1408351836283638318
:1054A0004FCF2B813C813FD12083318349CF37D1EE
:1054B0000D91119625D10A8B2E0103E115D1E0C083
:1054C0002ED16D907D901CD1062D072921F400E886
:1054D000602E04E2702E992022F400E1802E07E273
:1054E000902E80E090E001C00196F30101913F0110
:1054F000002319F088159905BCF30CD1230191956F
:1055000081959040680E791EBBC00E81002331F05A
:10551000082D092919F49924882483940FE814E2AA
:10552000088B198B0881003739F4F9D0ECD000E1F1
:10553000D5D000E0098330C0F1D046F40D911D9123
:105540002D913D91DDD0C801D90101C0DCD0088189
:105550000F3611F408E0ECCF053749F70AE0E8CF41
:10556000DDD04D915D9126F46D917D91C9D005C03E
:10557000C7D0652F660F660B762FCA01DB01772334
:105580004AF40DE209839095A095B09581959F4FBF
:10559000AF4FBF4F0AE0A2D03E0107E9600E00E026
:1055A000701E2E0107E9A0D0082F092B0A2B0B2B08
:1055B00011F001E001C000E00D83082D092919F464
:1055C0000D8100FF1FC094D0E889F989E00DF11D1D
:1055D0000081F30102933F018BD0C801D901012B57
:1055E000022B032B81F799206AF40F81002351F0DD
:1055F000A3D010E04501801A910A04C000E3F30132
:1056000002933F018E0109561F4F0619170908150D
:105610001905A4F30E81002399F10D8100FF30C01C
:105620000881083711F0083549F474D0F301088176
:10563000008370D000E3F301008322C00F3601F530
:10564000F30100810033E1F000E302933F0118C051
:1056500000EA602E04E2702E462C502EF2010081EA
:10566000002371F001E040D0F9CF0FEFC00ED01E43
:1056700003EC602E04E2702E06EC402E04E2502E65
:10568000420186189708A814B9041CF480E090E041
:1056900007C052D0A818B90810E0A01AB10AC50175
:1056A0000A81002321F401C063D00197EAF7098140
:1056B000002339F055D004C053D0F30101913F01CC
:1056C0005AD00FEF800E901EBAF70A81002309F41A
:1056D00037CE01970AF434CE4BD0FBCF10E00C87C5
:1056E0001D871E871F870895400E00E0501E0895F5
:1056F0004C855D856E857F858C019D010C942F26E0
:10570000A083B18308958D919D91A083B183A0E082
:10571000B0E008950FEF600E701E089580FBF70152
:10572000A081B1810895F701A081B1810D911D91F2
:10573000A083B183F80108950981002311F001E0ED
:10574000089500E00895F60100810895F6010081B2
:1057500000530A300895F60101916F0108830895FE
:1057600028853985089501E0C00E00E0D01E089517
:105770002885398500E2EA85FB8509950B811C8126
:105780000F5F1F4F0B831C8308950E94F028C801F0
:10579000D9011A013F7740E856E968E17BE40E94AD
:1057A0008E2838F416D0B38300E010E020E030E01B
:1057B0000DC03B2F0E94C1260E94B4260AD033831D
:1057C000A801B9018C019D010E945727E4E00C94C7
:1057D0000129F10100831183228308950E94E428A6
:1057E000C801D901BF7741E050E060E87FE33B2F7B
:1057F0000E94762870F440E00E946C2829F40BED9A
:105800001FE029E43FE350C0CC24DD24EE24FF2434
:105810001CC00BEDC02E0FE0D02E09E4E02EF72EB9
:1058200040E07FEB082F48D02801390140E050E0EC
:1058300060E87FE38C019D013FD0A801B90182019E
:1058400093010E94ED27C801D901AC01BD018C0173
:105850009D012DD02801390144E25FEF6BE27CEB22
:1058600026D048E854E466EA7EE328D048E150ECCC
:105870006FE370E423D045EB1CD0480159014AEE98
:1058800054EB66E870E48201930118D046EB11D026
:10589000A801B901840195010E94ED27AC01BD0169
:1058A00006D0A601B70108D0E0E10C94F5280C94CD
:1058B00074275DEF68E670E40C941327FDDFA20106
:1058C000B301F5CF20E006D0E9F70895259102D085
:1058D000E9F708952D9301501040202F212B0895B2
:1058E0008AE99BE5FC0105911491FC013296A59192
:1058F000B491FC01349625913491422F432B19F039
:10590000F901E4DF01C0DEDF06961BE5863A910768
:1059100048F3089540E00C948D2C0E94EC282897C1
:10592000802FB32F442E40E050E060E070E00E94F2
:10593000762810F401E001C000E0000F400EBF77B0
:1059400043E859EF62E27FE3082F3B2F80D076D007
:1059500041E05CEF6FE777E40E948E2888F5AE01A6
:105960000E94C52B6BD0042D10E06BD0488159816B
:105970006A817B8172D0088319832A833B83AE01BD
:105980004C5F5F4F2A0140E050E060E87EE35FD06B
:10599000A2010E94C52B40E050E060E870E40C8159
:1059A0001D812E813F8153D0A801B9010881198141
:1059B0002A813B810E9457270E94C126402E0CC09D
:1059C0000E94C126602E3DD0A801B9018C019D0125
:1059D00033D0460C03E0402240FA3EF4AC01BD0156
:1059E00000E010E020E83FE327D002E0401608F096
:1059F000B0588C019D0129D0280139014BEF57ED9A
:105A00006EE179E324D045E656E269E97BEB21D0EB
:105A100048E554E363EA7DE31CD041EE5DE565E2D1
:105A20007FEB17D04BED5FE069EC7FE316D00DD034
:105A30002896E8E00C94FD280E945727C801D90158
:105A4000089520E030E00C94BF26AC01BD010C9419
:105A5000742703D0A201B301FACF0C9413271B2F94
:105A60006A2FF901A081B181AD014F5F5F4F408383
:105A700051830C93A62FB12F0895BA93AA9324971C
:105A80000A831B8389019E012A5F3F4F2883398344
:105A9000BE01AE014E5F5F4F2FE23DE20E948F29B3
:105AA00020E0AA81BB812C932496A991B9910895F5
:105AB0000E94E82822974801590141E050E060E047
:105AC00070E00E94762898F440E00E946C2829F447
:105AD00000E010E020E030E04EC001E2ECEEF7E242
:105AE000008351830FEF1FEF2FE73FE744C0AE0164
:105AF0000E948325C801D90145EC53E062E47FE3AD
:105B00000E9413274AE151E562E17FE33BD0A801FF
:105B1000B9018C019D013BD0402E088100FF14C0CB
:105B20000A952DD0802F43EF54E065EB7FE3042DE1
:105B30000E94742737FB220F331F380F36952795A5
:105B400037F9C801D9010BC01AD0842D912FD90182
:105B500037FBAA0FBB1FB00FB695A795B7F940E06A
:105B600050E060E87EE38C019D010CD0AC01BD01EA
:105B7000840195010CD02296ECE00C94F92842E0C7
:105B80000C94AF250E9474272801390108950E94C2
:105B9000ED27A201B3010C941327A3032421A65BD4
:105BA0002703C72400002D20504C45415345205762
:105BB000414954202D2000202020202020203C3E40
:105BC000202020202020200045726173696E67200C
:105BD000454550524F4D2100726164696F646F6D8D
:105BE0002E75636F7A2E727500204B504F54322DF4
:105BF000584D2D762E3131272000202020202020C6
:105C00002020202020202020202000202050726FE3
:105C100066696C65203D2025642020002A2A2A2AF6
:105C2000204B553D2564202A2A2A2A2A002A2A2A7E
:105C30002A2A2A2A2A2A2A2A2A2A2A2A2A00545896
:105C4000202564487A202025646D41202000525888
:105C50002025646D5620202020004761696E3D2577
:105C60006420005458202D204572726F722121212A
:105C7000202020005258202D204572726F72212161
:105C80002120202000202020202020202020002053
:105C90002564256446256425630025642C2564203D
:105CA000002B253032645B00253032645B0023001A
:105CB0005D532564256446256425630025642C25F1
:105CC0006456200025646D5620005572783D256489
:105CD0006D5620202E2E2E2E2E2E20002A5A657232
:105CE0006F5F416463203C25643E202020005562A4
:105CF00061743D25642E256456202E2E2E2E2E2EC8
:105D00002000506F7765725F42617420203C2564EB
:105D10003E200025646D41202020202020202020CE
:105D200020202020200028256C642C256C64292E3E
:105D30002E2E20002A467265715F545820256C640F
:105D4000487A200025646D56202020202020002045
:105D5000413D2564202020002A436F696C20626C3D
:105D60002E2025633D256425632020002A46657288
:105D70007269746520200025633D25642563202019
:105D80000047726F756E6420626C2E20002B2564B4
:105D900020202020002D2E2E2E2E2E2E2E2E2B00BB
:105DA000566F6C756D65202020202020202020203B
:105DB000002564746F6E6520004265657073202055
:105DC00020202020202020202000256420202020AA
:105DD000202D2E2E2E2E2E2E2E2E2B00496E646957
:105DE000632E2020202020202020202020002B2572
:105DF00064202020202D2E2E2E2E2E2E2E2E2B00F7
:105E0000436F6E74722E202020202020202020201E
:105E1000200025646D412000506F7765722E202090
:105E20002020202020202020004761696E20202093
:105E30002020202020202020200038363432302F0F
:105E40003031323334353637383900202020282598
:105E5000303264293C253032643E2020202020004E
:105E600047726F756E6420626C2E2D4572726F7270
:105E70000047726F756E6420626C2E202D4F4B2D83
:105E8000200020202A2A2A202564202A2A2A2020AD
:105E90002020002B30305B200020204E6F204665F4
:105EA000727269746521202020002054616B652086
:105EB0004665727269746521202000202020202010
:105EC0004572726F72212020202020002020202087
:105ED00020204F4B21202020202020200020202087
:105EE0002020206C6F6E6720202020202020002C96
:105EF0000130313233343536373839414243444545
:105F00004600286E756C6C20706F696E746572291E
:105F10000030313233343536373839616263646585
:105F20006600464C4F4154533F2077726F6E672096
:105F3000666F726D617474657220696E7374616CE2
:095F40006C656421003F3F3F0045
:0400000300000000F9
:00000001FF
